
 Start  Stop   Length Name               Class

 00000H 063DBH 063DCH OBJECT1            DATA
 063E0H 063E0H 00000H DISKDATA           DATA
 163E0H 275BFH 111E0H SONGDATA           DATA
 275C0H 36FBFH 0FA00H PATTERNDATA        DATA
 36FC0H 3D01FH 06060H SCREENDATA         DATA
 3D020H 3D34BH 0032CH INFOLINE           CODE
 3D34CH 459B2H 08667H DISK               CODE
 459B3H 466CBH 00D19H SCREEN             CODE
 466D0H 475C6H 00EF7H MOUSE              CODE
 475C8H 47936H 0036FH MAIN               CODE
 47937H 484B9H 00B83H STARTUP            CODE
 484BAH 4DE41H 05988H PATTERN            CODE
 4DE44H 5B402H 0D5BFH MUSIC              CODE
 5B403H 5B899H 00497H GLBL               CODE
 5B89AH 5D736H 01E9DH INFOPAGE           CODE
 5D738H 5DB2BH 003F4H EMS                CODE
 5DB2CH 5DCDAH 001AFH ERROR              CODE
 5DCDCH 61361H 03686H INST               CODE
 61362H 6315BH 01DFAH FUNCTIONS          CODE
 6315CH 654E3H 02388H HELP               CODE
 654E4H 65FD0H 00AEDH KEYBOARD           CODE
 65FE0H 6681DH 0083EH MMTSR              CODE
 6681EH 68BB0H 02393H MESSAGE            CODE
 68BB1H 68E26H 00276H VESA               CODE
 68E30H 69E2FH 01000H STACKSEG           STACK


Detailed map of segments

 0000:0000 0000 C=DATA   S=OBJECT1        G=(none) M=IT.ASM     ACBP=29
 0000:0000 0000 C=DATA   S=OBJECT1        G=(none) M=IT_DISK.ASM ACBP=29
 0000:0000 0000 C=DATA   S=OBJECT1        G=(none) M=IT_DISPL.ASM ACBP=28
 0000:0000 0000 C=DATA   S=OBJECT1        G=(none) M=IT_EMS.ASM ACBP=29
 0000:0000 0000 C=DATA   S=OBJECT1        G=(none) M=IT_F.ASM   ACBP=29
 0000:0000 0000 C=DATA   S=OBJECT1        G=(none) M=IT_G.ASM   ACBP=28
 0000:0000 0000 C=DATA   S=OBJECT1        G=(none) M=IT_H.ASM   ACBP=29
 0000:0000 0000 C=DATA   S=OBJECT1        G=(none) M=IT_I.ASM   ACBP=29
 0000:0000 0000 C=DATA   S=OBJECT1        G=(none) M=IT_M.ASM   ACBP=28
 0000:0000 0000 C=DATA   S=OBJECT1        G=(none) M=IT_NET.ASM ACBP=29
 0000:0000 63DC C=DATA   S=OBJECT1        G=(none) M=IT_OBJ1.ASM ACBP=28
 0000:63DC 0000 C=DATA   S=OBJECT1        G=(none) M=IT_PE.ASM  ACBP=29
 0000:63DC 0000 C=DATA   S=OBJECT1        G=(none) M=IT_FOUR.ASM ACBP=29
 063E:0000 00010000 C=DATA   S=DISKDATA       G=(none) M=IT_DISK.ASM ACBP=6B
 163E:0000 0000 C=DATA   S=DISKDATA       G=(none) M=IT_I.ASM   ACBP=69
 163E:0000 0000 C=DATA   S=DISKDATA       G=(none) M=IT_NET.ASM ACBP=69
 163E:0000 0000 C=DATA   S=DISKDATA       G=(none) M=IT_FOUR.ASM ACBP=69
 163E:0000 0000 C=DATA   S=SONGDATA       G=(none) M=IT_MUSIC.ASM ACBP=69
 163E:0000 0000 C=DATA   S=SONGDATA       G=(none) M=IT_NET.ASM ACBP=69
 163E:0000 000111E0 C=DATA   S=SONGDATA       G=(none) M=IT_MDATA.ASM ACBP=68
 275C:0000 FA00 C=DATA   S=PATTERNDATA    G=(none) M=IT_PE.ASM  ACBP=69
 36FC:0000 6060 C=DATA   S=SCREENDATA     G=(none) M=IT_S.ASM   ACBP=69
 3D02:0000 0000 C=CODE   S=INFOLINE       G=(none) M=IT.ASM     ACBP=28
 3D02:0000 032C C=CODE   S=INFOLINE       G=(none) M=IT_L.ASM   ACBP=A8
 3D34:000C 0000 C=CODE   S=DISK           G=(none)    M=IT.ASM     ACBP=28
 3D34:000C 77B1 C=CODE   S=DISK           G=(none)    M=IT_DISK.ASM ACBP=28
 3D34:77BD 0000 C=CODE   S=DISK           G=(none)    M=IT_F.ASM   ACBP=29
 3D34:77C0 0EB3 C=CODE   S=DISK           G=(none)    M=IT_NET.ASM ACBP=A8
 3D34:8673 0000 C=CODE   S=DISK           G=(none)    M=IT_PE.ASM  ACBP=29
 459B:0003 0000 C=CODE   S=SCREEN         G=(none)  M=IT.ASM     ACBP=29
 459B:0003 0000 C=CODE   S=SCREEN         G=(none)  M=IT_F.ASM   ACBP=29
 459B:0003 0D19 C=CODE   S=SCREEN         G=(none)  M=IT_S.ASM   ACBP=28
 466D:0000 0000 C=CODE   S=MOUSE          G=(none)   M=IT.ASM     ACBP=29
 466D:0000 0000 C=CODE   S=MOUSE          G=(none)   M=IT_S.ASM   ACBP=29
 466D:0000 0EF7 C=CODE   S=MOUSE          G=(none)   M=IT_MOUSE.ASM ACBP=68
 475C:0008 0000 C=CODE   S=MAIN           G=(none)    M=IT.ASM     ACBP=A8
 475C:0008 036F C=CODE   S=MAIN           G=(none)    M=IT_M.ASM   ACBP=A8
 4793:0007 0B83 C=CODE   S=STARTUP        G=(none) M=IT.ASM     ACBP=28
 484B:000A 0000 C=CODE   S=PATTERN        G=(none) M=IT_DISK.ASM ACBP=29
 484B:000A 0000 C=CODE   S=PATTERN        G=(none) M=IT_DISPL.ASM ACBP=48
 484B:000A 0000 C=CODE   S=PATTERN        G=(none) M=IT_F.ASM   ACBP=29
 484B:000A 0000 C=CODE   S=PATTERN        G=(none) M=IT_G.ASM   ACBP=28
 484B:000A 0000 C=CODE   S=PATTERN        G=(none) M=IT_I.ASM   ACBP=29
 484B:000A 0000 C=CODE   S=PATTERN        G=(none) M=IT_NET.ASM ACBP=28
 484B:000A 5988 C=CODE   S=PATTERN        G=(none) M=IT_PE.ASM  ACBP=48
 4DE4:0004 0000 C=CODE   S=MUSIC          G=(none)   M=IT_DISK.ASM ACBP=29
 4DE4:0004 0000 C=CODE   S=MUSIC          G=(none)   M=IT_F.ASM   ACBP=29
 4DE4:0004 D5BF C=CODE   S=MUSIC          G=(none)   M=IT_MUSIC.ASM ACBP=A8
 4DE4:D5C3 0000 C=CODE   S=MUSIC          G=(none)   M=IT_NET.ASM ACBP=28
 5B40:0003 0000 C=CODE   S=GLBL           G=(none)    M=IT_DISPL.ASM ACBP=28
 5B40:0003 0497 C=CODE   S=GLBL           G=(none)    M=IT_G.ASM   ACBP=28
 5B40:049A 0000 C=CODE   S=GLBL           G=(none)    M=IT_L.ASM   ACBP=29
 5B89:000A 1B7C C=CODE   S=INFOPAGE       G=(none) M=IT_DISPL.ASM ACBP=28
 5B89:1B86 0321 C=CODE   S=INFOPAGE       G=(none) M=IT_FOUR.ASM ACBP=28
 5D73:0008 03F4 C=CODE   S=EMS            G=(none)     M=IT_EMS.ASM ACBP=48
 5DB2:000C 01AF C=CODE   S=ERROR          G=(none)   M=IT_ERR.ASM ACBP=28
 5DCD:000C 0000 C=CODE   S=INST           G=(none)    M=IT_F.ASM   ACBP=29
 5DCD:000C 0000 C=CODE   S=INST           G=(none)    M=IT_G.ASM   ACBP=28
 5DCD:000C 3686 C=CODE   S=INST           G=(none)    M=IT_I.ASM   ACBP=48
 5DCD:3692 0000 C=CODE   S=INST           G=(none)    M=IT_PE.ASM  ACBP=29
 6136:0002 1DFA C=CODE   S=FUNCTIONS      G=(none) M=IT_F.ASM   ACBP=28
 6315:000C 2388 C=CODE   S=HELP           G=(none)    M=IT_H.ASM   ACBP=28
 654E:0004 0AED C=CODE   S=KEYBOARD       G=(none) M=IT_K.ASM   ACBP=28
 65FE:0000 083E C=CODE   S=MMTSR          G=(none)   M=IT_MMTSR.ASM ACBP=68
 6681:000E 2393 C=CODE   S=MESSAGE        G=(none) M=IT_MSG.ASM ACBP=28
 68BB:0001 0276 C=CODE   S=VESA           G=(none)    M=IT_VESA.ASM ACBP=28
 68E3:0000 1000 C=STACK  S=STACKSEG       G=(none) M=IT.ASM     ACBP=75

  Address         Publics by Name

 466D:00DCA       ADDMOUSEQUEUE
 484B:002D8       AMPLIFICATION
 484B:00030       BASEOCTAVE
 484B:00D78       CENTRALISECURSOR
 459B:006A3       CHARACTERGENERATIONOFFSET
 3D02:00243       CLEARINFOLINE
 466D:00EDA       CMDLINEDISABLEMOUSE
 484B:00D77       COMMANDTOVALUE
 4793:00A9F       CRASHRECOVERY
 5B40:00003       CURRENTMODE
 4DE4:00352       CURRENTPATTERN
 3D34:00010       DISKDATAAREA
 3D34:00F34       DISKOPTIONS
 5B89:01881       DISPLAYMINUS
 5B89:01878       DISPLAYPLUS
 5B89:01A40       DISPLAYUPDATESCREEN
 5B89:01AAC       DISPLAY_GETDISPLAYWINDOWDATA
 5B89:01B11       DISPLAY_SELECTDISPLAYLIST
 4793:00B0F       DOSSHELL
 5B89:0179F       DRAWDISPLAYDATA
 466D:00B86       DRAWMOUSE
 3D34:06753       D_CLEARFILENAME
 3D34:03466       D_CLEARFILESPECIFIER
 3D34:06403 idle  D_DELETESAMPLEFILE
 3D34:0676E       D_DISABLEFILECOLOURS
 3D34:016CD       D_DRAWDIRECTORYWINDOW
 3D34:0173D       D_DRAWDRIVEWINDOW
 3D34:014B0       D_DRAWFILEWINDOW
 3D34:069D1       D_DRAWLOADINSTRUMENT
 3D34:04355       D_DRAWLOADSAMPLEWINDOW
 3D34:0755A       D_DRAWTIMER
 3D34:065AE       D_DRAWWAVEFORM
 3D34:0741A       D_GETFILENAME
 3D34:06768       D_GETFORMATTYPE
 3D34:0509B       D_GETLOADSAMPLEVARS
 3D34:073FE       D_GETPRESHELLDIRECTORY
 3D34:050AF       D_GOTOSTARTINGDIRECTORY
 3D34:010A6       D_INITDISK
 3D34:0684F       D_INITLOADINSTRUMENTS
 3D34:01469       D_INITLOADMODULE
 3D34:040E4       D_INITLOADSAMPLES
 3D34:04750       D_LIDRAWDRIVEWINDOW
 3D34:047A9       D_LIPOSTDRIVEWINDOW
 3D34:04787       D_LIPREDRIVEWINDOW
 3D34:02ADC       D_LOAD669
 3D34:0696A       D_LOADINSTRUMENTNAMES
 3D34:02EC0       D_LOADIT
 3D34:02C3D       D_LOADMOD
 3D34:0259C       D_LOADMTM
 3D34:0283A       D_LOADS3M
 3D34:05037       D_LOADSAMPLENAMES
 3D34:01858       D_LOADSONGNAMES
 3D34:0214E       D_LOADXM
 3D34:06018       D_LSCHECKLOOPVALUES
 3D34:06049       D_LSCHECKSUSLOOPVALUES
 3D34:046C7       D_LSDRAWDRIVEWINDOW
 3D34:0473F       D_LSPOSTDRIVEWINDOW
 3D34:0471B       D_LSPREDRIVEWINDOW
 3D34:0344A       D_NEWDIRECTORY
 3D34:033BB       D_NEWSPECIFIER
 3D34:03321       D_POSTDIRECTORYWINDOW
 3D34:03399       D_POSTDRIVEWINDOW
 3D34:0322D       D_POSTFILELOADWINDOW
 3D34:031EE       D_POSTFILESAVEWINDOW
 3D34:03298 idle  D_POSTFILEWINDOW
 3D34:06B4F       D_POSTLOADINSTRUMENT
 3D34:0462D       D_POSTLOADSAMPLEWINDOW
 3D34:033AA       D_POSTSAVEDRIVEWINDOW
 3D34:074FC       D_POSTTIMERLIST
 3D34:046B7       D_POSTVIEWSAMPLELIBRARY
 3D34:018C8       D_PREDIRECTORYWINDOW
 3D34:018EE       D_PREDRIVEWINDOW
 3D34:01889       D_PREFILEWINDOW
 3D34:06B22       D_PRELOADINSTRUMENT
 3D34:045FE       D_PRELOADSAMPLEWINDOW
 3D34:07420       D_RESETTIMER
 3D34:0740D       D_RESTOREPRESHELLDIRECTORY
 3D34:050BA       D_SAVEDIRECTORYCONFIGURATION
 3D34:062BC       D_SAVEINSTRUMENT
 3D34:03617       D_SAVEIT
 3D34:0347B       D_SAVEMODULE
 3D34:06166       D_SAVERAWSAMPLE
 3D34:03AD6       D_SAVES3M
 3D34:06100       D_SAVESAMPLE
 3D34:0607A       D_SAVESONG
 3D34:0620D       D_SAVEST3SAMPLE
 3D34:07416       D_SETDRIVEDIRECTORYFAR
 3D34:07451       D_SHOWTIME
 3D34:07712       D_SLOWINSTRUMENTSORT
 3D34:07670       D_SLOWSAMPLESORT
 3D34:01292       D_UNINITDISK
 3D34:06B60       D_VIEWINSTRUMENT
 0000:01016       EMSERRORVALUE
 0000:01014       EMSERRORVALUE2
 0000:01012       EMSERRORVALUE3
 0000:0100E       EMSERRORVALUE4
 0000:0100C       EMSERRORVALUE5
 0000:0100A       EMSERRORVALUE6
 0000:01008       EMSERRORVALUE7
 0000:01010       EMSERRORVALUE8
 5DB2:0018F       ERROR_INITHANDLER
 5DB2:001AA       ERROR_UNINITHANDLER
 5D73:001FD       E_ALLOCATEBLOCKEMS
 5D73:00374       E_ALLOCATEEMS
 5D73:003BA       E_EMSAVAILABLE
 5D73:001D5       E_GETEMSPAGEFRAME
 5D73:003F2       E_GETEMSVERSION
 5D73:000EB       E_GETFREEEMS
 5D73:003F7       E_GETINTERNALEMSHANDLE
 5D73:0002A       E_INITEMS
 5D73:001DA       E_MAPALIGNEDBLOCKEMS
 5D73:00180       E_MAPAVAILABLEEMSMEMORY
 5D73:0019B       E_MAPEMSMEMORY
 5D73:002E7       E_RELEASEBLOCKEMS
 5D73:00109       E_RELEASEEMS
 5D73:003DC       E_RESTOREEMSPAGEFRAME
 5D73:003C1       E_SAVEEMSPAGEFRAME
 5D73:001C4       E_UNINITEMS
 484B:00D7B       FASTVOLUMEAMPLIFICATION
 3D34:00066       FILENAME
 3D34:000C4       FILESPECIFIER
 484B:00D7D       FLAGS
 466D:00EE2       FORCEMOUSERESTORE
 5B89:01C8A       FOURIER_CHANGEPALETTE
 5B89:01B86       FOURIER_CREATETABLE
 5B89:01DA5       FOURIER_DRAWSCREEN
 5B89:01E96       FOURIER_IDLELIST
 5B89:01E9A       FOURIER_POSTFUNCTION
 5B89:01DA2       FOURIER_PREDRAWSCREEN
 5B89:01D40       FOURIER_START
 5B89:01BB1       FOURIER_TRANSFORM
 6136:01C35       F_CALCULATELENGTH
 6136:00369       F_CALLFARFUNCTION
 6136:00363       F_CALLFARPOSTFUNCTION
 6136:0035F       F_CALLFARPREFUNCTION
 6136:003E0       F_CHARACTERDEFINITIONS
 6136:0195C       F_CONFIGBUTTONSETUP
 6136:01518       F_DRAW3NUM
 6136:01700       F_DRAW5NUM
 6136:0036D       F_DRAWBOXOBJECT
 6136:00427       F_DRAWBUTTONOBJECT
 6136:018B8       F_DRAWHEADER
 6136:00D61       F_DRAWINFOLINE
 6136:008D6       F_DRAWSCALABLETHUMBBAR
 6136:0191D       F_DRAWSMCCHANNELS
 6136:00F92       F_DRAWSTRINGINPUT
 6136:00383       F_DRAWTEXTOBJECT
 6136:0080B       F_DRAWTHUMBBAR
 6136:01346       F_DRAWTOGGLE
 6136:01C4C       F_DRIVERSCREEN
 6136:01D44       F_FILEDOSSHELL
 6136:01CF4       F_FILELOAD
 6136:01CE0       F_FILEMENU
 6136:01D06       F_FILENEW
 6136:01D5B       F_FILEQUIT
 6136:01D32       F_FILESAVEAS
 6136:01D1B       F_FILESAVECURRENT
 6136:010E1       F_GOTOEMPTYLIST
 6136:01B91       F_HELP
 6136:01BB7       F_INFOPAGE
 6136:00344       F_INSTRUMENTBUTTONHANDLER
 6136:01CAA       F_INSTRUMENTLIBRARY
 6136:01C98       F_INSTRUMENTLIST
 6136:01C72       F_INSTRUMENTMENU
 6136:01B44       F_MAINMENU
 6136:01B84       F_MESSAGEEDITOR
 6136:01DB2       F_MIDI_DOWN
 6136:01DDC       F_MIDI_PGDN
 6136:01DC4       F_MIDI_PGUP
 6136:01D99       F_MIDI_UP
 6136:01A9E       F_NEWSONG
 6136:00341       F_NOTHING
 6136:01BA3       F_PLAYBACKMENU
 6136:01BFF       F_PLAYMARK
 6136:01BED       F_PLAYORDER
 6136:01BDB       F_PLAYPATTERN
 6136:01BC9       F_PLAYSONG
 6136:015B1       F_POST3NUM
 6136:01798       F_POST5NUM
 6136:00505       F_POSTBUTTONOBJECT
 6136:003C8       F_POSTEXITOBJECT
 6136:00B22       F_POSTSCALABLETHUMBBAR
 6136:0102A       F_POSTSTRINGINPUT
 6136:00B6E       F_POSTTHUMBBAR
 6136:013EF       F_POSTTOGGLE
 6136:01592       F_PRE3NUM
 6136:01779       F_PRE5NUM
 6136:004CC       F_PREBUTTONOBJECT
 6136:00A71       F_PRESCALABLETHUMBBAR
 6136:01006       F_PRESTRINGINPUT
 6136:009BF       F_PRETHUMBBAR
 6136:013BC       F_PRETOGGLE
 6136:00DE8       F_REDRAWSCREEN
 6136:01C23       F_REINITSOUNDCARD
 6136:01CBC       F_RELOADGRAVIS
 6136:01A96       F_RESET5NUMINPUTPOS
 6136:00DEC       F_RETURN0
 6136:00EDD       F_RETURN1
 6136:00DF9       F_RETURN192
 6136:00DF2       F_RETURN64
 6136:01CCE       F_SAMPLELIBRARY
 6136:01C86       F_SAMPLELIST
 6136:01C5E       F_SAMPLEMENU
 6136:01A86       F_SETAMIGA
 6136:019DF       F_SETCONTROLINSTRUMENT
 6136:019CF       F_SETCONTROLSAMPLE
 6136:003D8       F_SETDIRECTMODE
 6136:01A76       F_SETLINEAR
 6136:01A61       F_SETMONO
 6136:01A4C       F_SETSTEREO
 6136:00DA6       F_SHOWCHANNELS
 6136:01D72       F_SHOWMIDIZXXINPUT
 6136:01C11       F_STOP
 6136:01B77       F_VIEWORDERPAN
 6136:01B5D       F_VIEWPATTERN
 6136:01B6A       F_VIEWVARIABLES
 4793:00ACB       GETENVIRONMENT
 466D:00DC5       GETKEYBOARDLOCK
 4793:00A28       GETSTARTUPKEYLIST
 3D02:00326       GETTIMERCOUNTER
 5B40:00341       GLBL_ALT_F1
 5B40:0034D       GLBL_ALT_F2
 5B40:00359       GLBL_ALT_F3
 5B40:00365       GLBL_ALT_F4
 5B40:00371       GLBL_ALT_F5
 5B40:0037D       GLBL_ALT_F6
 5B40:00389       GLBL_ALT_F7
 5B40:00395       GLBL_ALT_F8
 5B40:0029A       GLBL_CTRL_F1
 5B40:002ED       GLBL_CTRL_F12
 5B40:002AD       GLBL_CTRL_F3
 5B40:002C5       GLBL_CTRL_F4
 5B40:002DD       GLBL_CTRL_F5
 5B40:0048C       GLBL_DRIVERSCREEN
 5B40:00231       GLBL_F10
 5B40:00256       GLBL_F11
 5B40:0025E       GLBL_F11_2
 5B40:00287       GLBL_F12
 5B40:00069       GLBL_F2
 5B40:00074       GLBL_F2_2
 5B40:000DC       GLBL_F3
 5B40:000F4       GLBL_F4
 5B40:00112       GLBL_F4_2
 5B40:00132       GLBL_F5
 5B40:00182       GLBL_F6
 5B40:00208       GLBL_F8
 5B40:00211       GLBL_F9
 5B40:0033C       GLBL_GETCURRENTMODE
 5B40:00300       GLBL_GETHEADERMODE
 5B40:003A1       GLBL_LEFTBRACE
 5B40:003C7       GLBL_LEFTSQUAREBRACKET
 5B40:001AF       GLBL_LOADINSTRUMENT
 5B40:00197       GLBL_LOADSAMPLE
 5B40:00411       GLBL_RESTOREMODE
 5B40:003B4       GLBL_RIGHTBRACE
 5B40:003DA       GLBL_RIGHTSQUAREBRACKET
 5B40:003ED       GLBL_SAVEMODE
 5B40:00337       GLBL_SETCURRENTMODE
 5B40:001C7       GLBL_SHIFT_F1
 5B40:001F2       GLBL_SHIFT_F6
 5B40:001DA       GLBL_SHIFT_F9
 5B40:00479       GLBL_TIMERSCREEN
 0000:01E1D       GLOBALKEYLIST
 0000:01E1E       HELPKEYVALUE
 6315:0228C       H_DRAWHELP
 6315:022FD       H_HELP
 6315:0232F       H_HELPDOWN
 6315:02377       H_HELPESC
 6315:0236D       H_HELPPGDN
 6315:0235A       H_HELPPGUP
 6315:0231F       H_HELPUP
 6315:0238C       H_SETHELPCONTEXT
 3D02:00227       IDLEUPDATEINFOLINE
 466D:00C8F       INITMOUSE
 3D02:00110       INITTIMERHANDLER
 5DCD:0000C       INSTRUMENTAMPLIFICATION
 3D34:00264       INSTRUMENTDIRECTORY
 5DCD:0013D       INSTRUMENTEDIT
 5DCD:0000E       INSTRUMENTSCREEN
 4793:00A23       ISSTARTUPKEYLIST
 5DCD:01AB6       I_AMPLIFYSAMPLE
 5DCD:01116       I_CALCULATEC5SPEED
 5DCD:019CF       I_CENTERSAMPLE
 5DCD:00E8D       I_CHECKLOOPVALUES
 5DCD:00ECB       I_CHECKSUSLOOPVALUES
 5DCD:01372 idle  I_CLEARSAMPLENAME
 5DCD:034BD       I_CLEARTABLES
 5DCD:01174       I_CONVERTSAMPLE
 5DCD:028EF       I_COPYINSTRUMENT
 5DCD:01320       I_CUTSAMPLE
 5DCD:0124F       I_CUTSAMPLEBEFORELOOP
 5DCD:0353D       I_DECREASEPLAYCHANNEL
 5DCD:01131       I_DELETEINSTRUMENT
 5DCD:010DE       I_DELETESAMPLE
 5DCD:027C1       I_DOUBLESAMPLESPEED
 5DCD:029F5       I_DRAWENVELOPE
 5DCD:01F7A       I_DRAWINSTRUMENTWINDOW
 5DCD:0233F       I_DRAWNOTEWINDOW
 5DCD:035A1       I_DRAWPITCHPANCENTER
 5DCD:00A71       I_DRAWSAMPLELIST
 5DCD:00F09       I_DRAWWAVEFORM
 5DCD:02781       I_EXCHANGEINSTRUMENTS
 5DCD:015D7       I_EXCHANGESAMPLES
 5DCD:00987       I_GETINSTRUMENTOFFSET
 5DCD:00981       I_GETINSTRUMENTSCREEN
 5DCD:0368C       I_GETPRESETENVELOPEOFFSET
 5DCD:0099A       I_GETSAMPLEOFFSET
 5DCD:027E1       I_HALVESAMPLESPEED
 5DCD:03635       I_IDLEUPDATEENVELOPE
 5DCD:03522       I_INCREASEPLAYCHANNEL
 5DCD:033D6       I_INSTRUMENTLISTNOTEOFF
 5DCD:033A9       I_INSTRUMENTLISTSPACE
 5DCD:011DC       I_INVERTSAMPLE
 5DCD:02B39       I_MAPENVELOPE
 5DCD:02157       I_PLAYNOTE
 5DCD:03505       I_PLAYSAMPLE
 5DCD:02A8D       I_POSTENVELOPE
 5DCD:021EA       I_POSTINSTRUMENTWINDOW
 5DCD:02437       I_POSTNOTEWINDOW
 5DCD:035E3       I_POSTPITCHPANCENTER
 5DCD:00BC3       I_POSTSAMPLELIST
 5DCD:02A85       I_PREENVELOPE
 5DCD:02035       I_PREINSTRUMENTWINDOW
 5DCD:023FB       I_PRENOTEWINDOW
 5DCD:035D3       I_PREPITCHPANCENTER
 5DCD:00B68       I_PRESAMPLELIST
 5DCD:0111A       I_PRINTC5FREQUENCY
 5DCD:0282E       I_REPLACEINSTRUMENT
 5DCD:016A0       I_REPLACESAMPLE
 5DCD:0196A       I_RESIZESAMPLE
 5DCD:01972       I_RESIZESAMPLENOINT
 5DCD:01BEE       I_REVERSESAMPLE
 5DCD:03675       I_SAMPLEBUTTONHANDLER
 5DCD:00D5D       I_SAMPLEDOWN
 5DCD:02813       I_SAMPLESPEEDSEMIDOWN
 5DCD:027F2       I_SAMPLESPEEDSEMIUP
 5DCD:00D7A       I_SAMPLEUP
 5DCD:028A5       I_SCALEINSTRUMENTVOLUMES
 5DCD:0285B       I_SCALESAMPLEVOLUMES
 5DCD:009C2       I_SELECTSCREEN
 5DCD:0343E       I_SHOWINSTRUMENTPLAY
 5DCD:00E25       I_SHOWSAMPLEINFO
 5DCD:033F2       I_SHOWSAMPLEPLAY
 5DCD:02917       I_SWAPINSTRUMENTS
 5DCD:0161C       I_SWAPSAMPLES
 5DCD:034CA       I_TAGINSTRUMENT
 5DCD:034D1       I_TAGSAMPLE
 5DCD:03589       I_TOGGLEMULTICHANNEL
 5DCD:01DA6       I_TOGGLESAMPLEQUALITY
 5DCD:02966       I_UPDATEINSTRUMENT
 654E:00966       K_CLEARKEYBOARDQUEUE
 654E:009A6       K_DRAWTABLES
 654E:0070B       K_GETKEY
 654E:005EA       K_INITKEYBOARD
 654E:00693       K_INSTALLDOSHANDLER
 654E:00A46       K_INSTALLKEYBOARDTYPE
 654E:00977       K_ISANYKEYDOWN
 654E:0098F       K_ISKEYDOWN
 654E:006D7       K_ISKEYWAITING
 654E:00A9B       K_REMOVEKEYBOARDTYPE
 654E:00996       K_RESETKEYBOARDTABLES
 654E:00AAD       K_SETSCROLLLOCK
 654E:00A23       K_SHOWMIDIINPUT
 654E:00651       K_UNINITKEYBOARD
 654E:006B3       K_UNINSTALLDOSHANDLER
 484B:00FEF       LASTINSTRUMENT
 484B:00086 idle  LASTKEYBOARD1
 0000:02184 idle  LOGOCHARACTER
 3D34:05FB5       LSWINDOW_DOWN
 3D34:05FA1       LSWINDOW_UP
 5DCD:00127       MAXNODE
 484B:00024       MAXROW
 484B:00D79       MIDIAMPLIFICATION
 654E:00AB6       MIDIBUFFEREMPTY
 484B:00D7A       MIDICENTRALNOTE
 4DE4:09966       MIDIDATAAREA
 654E:00ABD       MIDISEND
 5DCD:0207B       MIDI_ALLOCATECHANNEL
 5DCD:020CD       MIDI_CLEARTABLE
 5DCD:020C3       MIDI_FINDCHANNEL
 5DCD:020BB       MIDI_GETCHANNEL
 5DCD:020E2       MIDI_NOTEOFF
 5DCD:0210F       MIDI_PLAYNOTE
 5DCD:034D8       MIDI_PLAYSAMPLE
 484B:056C4       MIDI_SETINSTRUMENT
 65FE:00001       MMTSR_INSTALLMMTSR
 65FE:0006F       MMTSR_UNINSTALLMMTSR
 484B:0060B       MODIFIED
 466D:00E3D       MOUSEADDEVENT
 466D:00000       MOUSECHARACTERGENERATIONOFFSET
 466D:00E61       MOUSECLEAREVENTS
 466D:00E73       MOUSEGETSTATUS
 466D:00DF5       MOUSEINPUT
 466D:00E6A       MOUSEREMOVEEVENTS
 466D:00D9B       MOUSERESTOREEVENTS
 466D:00D76       MOUSESAVEEVENTS
 466D:00CF1       MOUSESECONDSETDISABLE
 466D:00CEA       MOUSESECONDSETENABLE
 466D:00D27       MOUSESETXY
 466D:00CF8       MOUSETOGGLE
 466D:00E86       MOUSEUPDATEDISABLE
 466D:00E7F       MOUSEUPDATEENABLE
 6681:01FE5       MSG_DRAWMESSAGE
 6681:0237D       MSG_GETMESSAGELENGTH
 6681:02392       MSG_GETMESSAGEOFFSET
 6681:020BE       MSG_POSTMESSAGE
 6681:0208F       MSG_PREMESSAGE
 6681:01FCB       MSG_RESETMESSAGE
 484B:00034       MULTICHANNELINFO
 4DE4:0BDDD       MUSIC_ALLOCATEPATTERN
 4DE4:0BEA5       MUSIC_ALLOCATESAMPLE
 4DE4:0D1D6       MUSIC_ASSIGNSAMPLETOINSTRUMENT
 4DE4:0C17E       MUSIC_AUTODETECTSOUNDCARD
 4DE4:0C056       MUSIC_CLEARALLINSTRUMENTS
 4DE4:0C001       MUSIC_CLEARALLSAMPLENAMES
 4DE4:0C034       MUSIC_CLEARINSTRUMENT
 4DE4:0BFDE       MUSIC_CLEARSAMPLENAME
 4DE4:0D165       MUSIC_DECREASESPEED
 4DE4:0D27F       MUSIC_DECREASEVOLUME
 4DE4:0D3B5       MUSIC_GETDELAY
 4DE4:0D1C5       MUSIC_GETDISPLAYVARIABLES
 4DE4:0D3A0       MUSIC_GETDRIVERSCREEN
 4DE4:0D3A5       MUSIC_GETDRIVERVARIABLE
 4DE4:0D336       MUSIC_GETFREESOUNDCARDMEMORY
 4DE4:0CF8F       MUSIC_GETHOSTCHANNELINFORMATIONTABLE
 4DE4:0C254       MUSIC_GETINSTRUMENTMODE
 4DE4:0D37C       MUSIC_GETLASTCHANNEL
 4DE4:0D546       MUSIC_GETMIDIDATAAREA
 4DE4:0CBEC       MUSIC_GETNUMBEROFINSTRUMENTS
 4DE4:0CBC4       MUSIC_GETNUMBEROFSAMPLES
 4DE4:0D33C       MUSIC_GETNUMCHANNELS
 4DE4:0BD38       MUSIC_GETPATTERN
 4DE4:0D518       MUSIC_GETPATTERNLENGTH
 4DE4:0BD80       MUSIC_GETPATTERNLOCATION
 4DE4:0BD89       MUSIC_GETPATTERNLOCATIONNOCOUNT
 4DE4:0D341       MUSIC_GETPITCHTABLE
 4DE4:0CC9A       MUSIC_GETPLAYMODE
 4DE4:0CCB2       MUSIC_GETPLAYMODE2
 4DE4:0CC22       MUSIC_GETSAMPLELOCATION
 4DE4:0CF95       MUSIC_GETSLAVECHANNELINFORMATIONTABLE
 4DE4:0C082       MUSIC_GETSONGSEGMENT
 4DE4:0BC51       MUSIC_GETWAVEFORM
 4DE4:0D14C       MUSIC_INCREASESPEED
 4DE4:0D263       MUSIC_INCREASEVOLUME
 4DE4:0D360       MUSIC_INITMIXTABLE
 4DE4:0BCAF       MUSIC_INITMUSIC
 4DE4:0D115       MUSIC_INITMUTETABLE
 4DE4:0D134       MUSIC_INITSTEREO
 4DE4:0CD6D       MUSIC_KBPLAYSONG
 4DE4:0CFCA       MUSIC_LASTORDER
 4DE4:0CF9E       MUSIC_NEXTORDER
 4DE4:0D35B       MUSIC_PATTERNSTORAGE
 4DE4:0CEB7       MUSIC_PLAYNOTE
 4DE4:0CD2C       MUSIC_PLAYPARTSONG
 4DE4:0CCCB       MUSIC_PLAYPATTERN
 4DE4:0CF39       MUSIC_PLAYSAMPLE
 4DE4:0CCF5       MUSIC_PLAYSONG
 4DE4:0BC61       MUSIC_POLL
 4DE4:0D298       MUSIC_REGETLOOPINFORMATION
 4DE4:0BC9F       MUSIC_REINITSOUNDCARD
 4DE4:0C023       MUSIC_RELEASEALLPATTERNS
 4DE4:0C012       MUSIC_RELEASEALLSAMPLES
 4DE4:0BCF4       MUSIC_RELEASEPATTERN
 4DE4:0BF62       MUSIC_RELEASESAMPLE
 4DE4:0D25C       MUSIC_REVERSECHANNELS
 4DE4:0D51D       MUSIC_SAVEMIDICONFIG
 4DE4:0D1BF       MUSIC_SETADDRESS
 4DE4:0D1AC       MUSIC_SETDMA
 4DE4:0D3AA       MUSIC_SETDRIVERVARIABLE
 4DE4:0D006       MUSIC_SETGLOBALVOLUME
 4DE4:0D1B9       MUSIC_SETIRQ
 4DE4:0D256       MUSIC_SETLIMIT
 4DE4:0D1B3       MUSIC_SETMIXSPEED
 4DE4:0D3AF       MUSIC_SETNEXTORDER
 4DE4:0D17E       MUSIC_SETSOUNDCARD
 4DE4:0D1A1       MUSIC_SETSOUNDCARDDRIVER
 4DE4:0C232       MUSIC_SHOWAUTODETECTSOUNDCARD
 4DE4:0D4FA       MUSIC_SHOWTIME
 4DE4:0D0B1       MUSIC_SOLOCHANNEL
 4DE4:0D2E5       MUSIC_SOUNDCARDLOADALLSAMPLES
 4DE4:0D2CE       MUSIC_SOUNDCARDLOADSAMPLE
 4DE4:0CDC0       MUSIC_STOP
 4DE4:0D421       MUSIC_TIMESONG
 4DE4:0D079       MUSIC_TOGGLECHANNEL
 4DE4:0D54C       MUSIC_TOGGLEORDERUPDATE
 4DE4:0D347       MUSIC_TOGGLEREVERSE
 4DE4:0D561       MUSIC_TOGGLESOLOINSTRUMENT
 4DE4:0D56C       MUSIC_TOGGLESOLOSAMPLE
 4DE4:0C061       MUSIC_UNINITMUSIC
 4DE4:0D0AA       MUSIC_UNMUTEALL
 4DE4:0CEAF       MUSIC_UPDATEPATTERNOFFSET
 475C:000F1       M_FUNCTIONDIVIDER
 475C:00169       M_FUNCTIONHANDLER
 475C:00363       M_OBJECT1LIST
 475C:00360       M_OBJECT1LISTDEFAULT
 3D34:085C9       NETWORK_ADDWORDTOQUEUE
 3D34:07B02       NETWORK_DRAWDRIVERSCREEN
 3D34:07A63       NETWORK_DRIVERSCREEN
 3D34:08613       NETWORK_ENSURENONETWORK
 3D34:08496       NETWORK_FINISHEDSENDQUEUE
 3D34:0846A       NETWORK_GETSENDQUEUE
 3D34:07D45       NETWORK_POLL
 3D34:07BD5       NETWORK_POSTDRIVERSCREEN
 3D34:07B7F       NETWORK_PREDRIVERSCREEN
 3D34:084D6       NETWORK_QUEUESAMPLEDATA
 3D34:08647       NETWORK_SENDINSTRUMENTHEADER
 3D34:08630       NETWORK_SENDSAMPLEHEADER
 3D34:0865E       NETWORK_SENDSONGDATAINFORMATION
 3D34:07D7B       NETWORK_SHUTDOWN
 3D34:085EF       NETWORK_UPDATEPATTERN
 3D34:085DA       NETWORK_UPDATEPATTERNIFIDLE
 466D:00E78       NEWCHARACTERSET
 5DCD:00121       NEWSAMPLESIZE
 5DCD:00135       NODEHELD
 484B:00026       NUMBEROFROWS
 0000:00000       O1_AUTODETECTLIST
 0000:00325       O1_C5FREQUENCYLIST
 0000:0373C       O1_CONFIGUREITLIST
 0000:05172       O1_CONFIGUREPALETTELIST
 0000:02608       O1_CONFIRMCLEARMESSAGE
 0000:024FA       O1_CONFIRMCONVERT2LIST
 0000:024E8       O1_CONFIRMCONVERTLIST
 0000:025D2       O1_CONFIRMCUTSAMPLE
 0000:02566       O1_CONFIRMDELETE
 0000:02578       O1_CONFIRMDELETE2
 0000:0258A       O1_CONFIRMDELETE3
 0000:025F6       O1_CONFIRMDELETEINSTRUMENT
 0000:025E4       O1_CONFIRMDELETESAMPLE
 0000:025C0       O1_CONFIRMDISCARDLIST
 0000:0261A       O1_CONFIRMNOSAVE
 0000:02542       O1_CONFIRMOVERWRITELIST
 0000:028F1       O1_CONFIRMQUIT
 0000:025AE       O1_CONFIRMRESAVELIST
 0000:0259C       O1_CONFIRMSAVERENAMELIST
 0000:02EA5       O1_COPYINSTRUMENTLIST
 0000:00365       O1_CRASHRECOVERY
 0000:046A3       O1_DISPLAYLIST
 0000:05128       O1_EDITSAMPLENAME
 0000:0082E       O1_EMPTYLIST
 0000:00335       O1_EMSWARNINGMESSAGE
 0000:0251E       O1_ENABLEINSTRUMENTMODE
 0000:02EB7       O1_EXCHANGEINSTRUMENTLIST
 0000:02E4B       O1_EXCHANGESAMPLELIST
 0000:04B7C       O1_FILEMENU
 0000:063A5       O1_FOURIERDISPLAY
 0000:046B7       O1_FULLDISPLAYLIST
 0000:002CD       O1_GETAMPLIST
 0000:002F9       O1_GETFASTAMPLIST
 0000:002E3       O1_GETINSTRUMENTAMPLIST
 0000:000BE       O1_HELPLIST
 0000:02554       O1_INITIALISEINSTRUMENTLIST
 0000:02530       O1_INITINSTRUMENT
 0000:03BC6       O1_INSTRUMENTLISTGENERAL
 0000:041E0       O1_INSTRUMENTLISTPANNING
 0000:043B8       O1_INSTRUMENTLISTPITCH
 0000:03F23       O1_INSTRUMENTLISTVOLUME
 0000:05071       O1_INSTRUMENTMENU
 0000:03B06       O1_KEYBOARDLIST
 0000:007FE       O1_LOAD669LIST
 0000:05A4C       O1_LOADINSTRUMENTLIST
 0000:00816       O1_LOADITLIST
 0000:007E6       O1_LOADMODLIST
 0000:006FA       O1_LOADMODULELIST
 0000:007CE       O1_LOADMTMLIST
 0000:00758       O1_LOADNETWORKDRIVER
 0000:0079E       O1_LOADS3MLIST
 0000:00373       O1_LOADSAMPLELIST
 0000:007B6       O1_LOADXMLIST
 0000:0026D       O1_LONGMESSAGELIST
 0000:04942       O1_MAINMENU
 0000:05B2B       O1_MESSAGELIST
 0000:05FBC       O1_MIDISCREEN
 0000:00345       O1_NETWORKERRORLIST
 0000:04731       O1_NEWSONGLIST
 0000:002AD       O1_NOBLOCKDATALIST
 0000:0022D       O1_NOBLOCKMARKEDLIST
 0000:0001E       O1_ORDERPANNINGLIST
 0000:0309C       O1_ORDERVOLUMELIST
 0000:0024D       O1_OUTOFMEMORYLIST
 0000:0027D       O1_OUTOFSAMPLESLIST
 0000:0023D       O1_OUTOFSOUNDCARDMEMORYLIST
 0000:0028D       O1_OVERLAPBLOCKLIST
 0000:000D4       O1_PATTERNEDITLIST
 0000:0025D       O1_PATTERNSIZEMISMATCHLIST
 0000:002BD       O1_PATTERNTOOLONGLIST
 0000:000E8       O1_PECONFIGLIST
 0000:04D0F       O1_PLAYBACKMENU
 0000:02E6F       O1_REPLACEINSTRUMENTLIST
 0000:02E5D       O1_REPLACESAMPLELIST
 0000:02EC9       O1_RESIZESAMPLELIST
 0000:0030F       O1_SAMPLEAMPLIFICATIONLIST
 0000:0250C       O1_SAMPLECENTERLIST
 0000:0068C       O1_SAMPLELIST
 0000:04F87       O1_SAMPLEMENU
 0000:0076E       O1_SAVEITLIST
 0000:00726       O1_SAVEMODULELIST
 0000:00786       O1_SAVES3MLIST
 0000:02903       O1_SELECTMULTICHANNEL
 0000:0011C       O1_SETPATTERNLENGTH
 0000:06378       O1_SHOWTIME
 0000:062E4       O1_STEREOSAMPLELIST
 0000:02E93       O1_SWAPINSTRUMENTLIST
 0000:0029D       O1_SWAPOUTOFRANGELIST
 0000:02E81       O1_SWAPSAMPLELIST
 0000:00355       O1_TEMPLATEERRORLIST
 0000:046EC       O1_THUMBSTRINGLIST
 0000:0626C       O1_TIMERLIST
 0000:028A2       O1_UNABLETOSAVELIST
 0000:05AF5       O1_UNDOLIST
 0000:05A7B       O1_VIEWINSTRUMENTLIBRARY
 0000:003B9       O1_VIEWSAMPLELIBRARY
 484B:0001A       ORDER
 0000:01E87       ORDERKEYVALUE
 459B:00028       PALETTEDEFS
 484B:0000A       PATTERNDATAAREA
 484B:0087E       PATTERNLENGTHEND
 484B:0087C       PATTERNLENGTHSTART
 484B:0060C       PATTERNMODIFIED
 484B:0001E       PATTERNNUMBER
 484B:0087A       PATTERNSETLENGTH
 484B:05625       PECHECKMODIFIED
 484B:02769       PEFUNCTION_DECREASEOCTAVE
 484B:05524       PEFUNCTION_DRAWUNDO
 484B:02779       PEFUNCTION_INCREASEOCTAVE
 484B:031B4       PEFUNCTION_OUTOFMEMORYMESSAGE
 484B:05577       PEFUNCTION_POSTUNDO
 484B:0555A       PEFUNCTION_PREUNDO
 484B:03A6D       PEFUNCTION_STORECURRENTPATTERN
 484B:05643       PERESETMODIFIED
 484B:054EB idle  PE_CLEARUNDOBUFFER
 484B:01054       PE_CONVAX2NUM
 484B:0513F       PE_DELETEINSTRUMENT
 484B:012E6       PE_DRAWORDERLIST
 484B:01673       PE_DRAWPATTERNEDIT
 484B:05372       PE_F7
 484B:011E0       PE_FILLHEADER
 484B:012C9       PE_FILLSPEEDTEMPO
 484B:046A4       PE_GETCURRENTPATTERN
 484B:04FBC       PE_GETLASTINSTRUMENT
 484B:0109C       PE_GETMAXORDER
 484B:011B9       PE_GETMAXPATTERN
 484B:0543D       PE_GETPATTERNCONFIGOFFSET
 484B:03A97       PE_GOTOPATTERN
 484B:015DB       PE_INITPATTERNEDIT
 484B:0508C       PE_INSERTINSTRUMENT
 484B:0597F       PE_NEWPATTERN
 484B:013BA       PE_POSTORDERLIST
 484B:01D00       PE_POSTPATTERNEDIT
 484B:01376       PE_PREORDERLIST
 484B:01B41       PE_PREPATTERNEDIT
 484B:0114E       PE_RESETORDERPATTERN
 484B:05966       PE_RESTORECURRENTPATTERN
 484B:058FC       PE_RESTOREMIDINOTE
 484B:05948       PE_SAVECURRENTPATTERN
 484B:02A4C       PE_SETCOMMANDCURSOR
 484B:05940       PE_SETPATTERNMODIFIED
 484B:052FE       PE_SHOWORDER
 484B:04FC4       PE_SWAPINSTRUMENTS
 484B:041C6       PE_TRANSLATE669PATTERN
 484B:058C0       PE_TRANSLATEMIDI
 484B:0414C       PE_TRANSLATEMODPATTERN
 484B:040EC       PE_TRANSLATEMTMPATTERN
 484B:042D9       PE_TRANSLATES3MPATTERN
 484B:03E98       PE_TRANSLATEXMPATTERN
 484B:015A4       PE_UNINITPATTERNEDIT
 484B:051ED       PE_UPDATEINSTRUMENTS
 5B89:0184A       POSTDISPLAYDATA
 4793:009C5       QUIT
 4793:00AF2       REFRESH
 475C:000F0       RELEASETIMESLICE
 466D:008C8       RESTOREMOUSE
 466D:00922       RESTOREMOUSEGRAPHICS
 484B:00CA8       ROWHILIGHT1
 484B:00CA9       ROWHILIGHT2
 5DCD:00145       SAMPLEAMPLIFICATION
 3D34:0021E       SAMPLEDIRECTORY
 3D34:002AB       SAMPLENAME
 5DCD:00011       SAMPLENUMBER
 5DCD:0011D       SAMPLENUMBERINPUT
 3D02:0024E       SETINFOLINE
 3D02:00264       SETINFOLINE2
 466D:00DC0       SETKEYBOARDLOCK
 466D:00E8D       SETMOUSECURSORTYPE
 3D02:000F8       SHOWUSAGETIME
 484B:00032       SKIPVALUE
 4DE4:09964       SONGDATAAREA
 3D34:001D8       SONGDIRECTORY
 3D02:00317       STARTCLOCK
 459B:00975       S_CLEARSCREEN
 459B:00CA5       S_DEFINEHIASCII
 459B:008B7       S_DEFINESMALLNUMBERS
 459B:00AA8       S_DIRECTDRAWSTRING
 459B:0098A       S_DRAWBOX
 459B:00C62       S_DRAWSMALLBOX
 459B:00ABD       S_DRAWSTRING
 459B:00BE2       S_GENERATECHARACTERS
 459B:00960       S_GETDESTINATION
 459B:00BD9       S_GETGENERATIONTABLEOFFSET
 459B:00C7E       S_GETPALETTEOFFSET
 459B:00A99       S_HILIGHT
 459B:006B7       S_INITSCREEN
 459B:00CE5       S_INVERTCURSOR
 459B:00871       S_REDEFINECHARACTERS
 459B:0084B       S_RESETSEQUENCER
 459B:0078C       S_RESTORESCREEN
 459B:0076A       S_SAVESCREEN
 459B:00A59       S_SETDIRECTMODE
 459B:007FD       S_SETPALETTE
 459B:007F9       S_SETPALETTE2
 459B:00825       S_SETSEQUENCER
 459B:0094F       S_UNINITSCREEN
 459B:009F8       S_UPDATESCREEN
 459B:00C84       S_USEPRESETPALETTE
 6136:000D8       THUMBSTRINGENTER
 466D:00CE5       UNINITMOUSE
 3D02:0012C       UNINITTIMERHANDLER
 3D02:00152       UPDATEINFOLINE
 5DCD:03671       UPDATEWAVEFORM
 68BB:00201       VESA_DETECT
 68BB:00244 idle  VESA_GETINFO
 68BB:0025B       VESA_SETBLOCK
 68BB:00221       VESA_SETMODE
 459B:006A5       VGAFLAGS

  Address         Publics by Value

 0000:063A5       O1_FOURIERDISPLAY
 0000:06378       O1_SHOWTIME
 0000:062E4       O1_STEREOSAMPLELIST
 0000:0626C       O1_TIMERLIST
 0000:05FBC       O1_MIDISCREEN
 0000:05B2B       O1_MESSAGELIST
 0000:05AF5       O1_UNDOLIST
 0000:05A7B       O1_VIEWINSTRUMENTLIBRARY
 0000:05A4C       O1_LOADINSTRUMENTLIST
 0000:05172       O1_CONFIGUREPALETTELIST
 0000:05128       O1_EDITSAMPLENAME
 0000:05071       O1_INSTRUMENTMENU
 0000:04F87       O1_SAMPLEMENU
 0000:04D0F       O1_PLAYBACKMENU
 0000:04B7C       O1_FILEMENU
 0000:04942       O1_MAINMENU
 0000:04731       O1_NEWSONGLIST
 0000:046EC       O1_THUMBSTRINGLIST
 0000:046B7       O1_FULLDISPLAYLIST
 0000:046A3       O1_DISPLAYLIST
 0000:043B8       O1_INSTRUMENTLISTPITCH
 0000:041E0       O1_INSTRUMENTLISTPANNING
 0000:03F23       O1_INSTRUMENTLISTVOLUME
 0000:03BC6       O1_INSTRUMENTLISTGENERAL
 0000:03B06       O1_KEYBOARDLIST
 0000:0373C       O1_CONFIGUREITLIST
 0000:0309C       O1_ORDERVOLUMELIST
 0000:02EC9       O1_RESIZESAMPLELIST
 0000:02EB7       O1_EXCHANGEINSTRUMENTLIST
 0000:02EA5       O1_COPYINSTRUMENTLIST
 0000:02E93       O1_SWAPINSTRUMENTLIST
 0000:02E81       O1_SWAPSAMPLELIST
 0000:02E6F       O1_REPLACEINSTRUMENTLIST
 0000:02E5D       O1_REPLACESAMPLELIST
 0000:02E4B       O1_EXCHANGESAMPLELIST
 0000:02903       O1_SELECTMULTICHANNEL
 0000:028F1       O1_CONFIRMQUIT
 0000:028A2       O1_UNABLETOSAVELIST
 0000:0261A       O1_CONFIRMNOSAVE
 0000:02608       O1_CONFIRMCLEARMESSAGE
 0000:025F6       O1_CONFIRMDELETEINSTRUMENT
 0000:025E4       O1_CONFIRMDELETESAMPLE
 0000:025D2       O1_CONFIRMCUTSAMPLE
 0000:025C0       O1_CONFIRMDISCARDLIST
 0000:025AE       O1_CONFIRMRESAVELIST
 0000:0259C       O1_CONFIRMSAVERENAMELIST
 0000:0258A       O1_CONFIRMDELETE3
 0000:02578       O1_CONFIRMDELETE2
 0000:02566       O1_CONFIRMDELETE
 0000:02554       O1_INITIALISEINSTRUMENTLIST
 0000:02542       O1_CONFIRMOVERWRITELIST
 0000:02530       O1_INITINSTRUMENT
 0000:0251E       O1_ENABLEINSTRUMENTMODE
 0000:0250C       O1_SAMPLECENTERLIST
 0000:024FA       O1_CONFIRMCONVERT2LIST
 0000:024E8       O1_CONFIRMCONVERTLIST
 0000:02184 idle  LOGOCHARACTER
 0000:01E87       ORDERKEYVALUE
 0000:01E1E       HELPKEYVALUE
 0000:01E1D       GLOBALKEYLIST
 0000:01016       EMSERRORVALUE
 0000:01014       EMSERRORVALUE2
 0000:01012       EMSERRORVALUE3
 0000:01010       EMSERRORVALUE8
 0000:0100E       EMSERRORVALUE4
 0000:0100C       EMSERRORVALUE5
 0000:0100A       EMSERRORVALUE6
 0000:01008       EMSERRORVALUE7
 0000:0082E       O1_EMPTYLIST
 0000:00816       O1_LOADITLIST
 0000:007FE       O1_LOAD669LIST
 0000:007E6       O1_LOADMODLIST
 0000:007CE       O1_LOADMTMLIST
 0000:007B6       O1_LOADXMLIST
 0000:0079E       O1_LOADS3MLIST
 0000:00786       O1_SAVES3MLIST
 0000:0076E       O1_SAVEITLIST
 0000:00758       O1_LOADNETWORKDRIVER
 0000:00726       O1_SAVEMODULELIST
 0000:006FA       O1_LOADMODULELIST
 0000:0068C       O1_SAMPLELIST
 0000:003B9       O1_VIEWSAMPLELIBRARY
 0000:00373       O1_LOADSAMPLELIST
 0000:00365       O1_CRASHRECOVERY
 0000:00355       O1_TEMPLATEERRORLIST
 0000:00345       O1_NETWORKERRORLIST
 0000:00335       O1_EMSWARNINGMESSAGE
 0000:00325       O1_C5FREQUENCYLIST
 0000:0030F       O1_SAMPLEAMPLIFICATIONLIST
 0000:002F9       O1_GETFASTAMPLIST
 0000:002E3       O1_GETINSTRUMENTAMPLIST
 0000:002CD       O1_GETAMPLIST
 0000:002BD       O1_PATTERNTOOLONGLIST
 0000:002AD       O1_NOBLOCKDATALIST
 0000:0029D       O1_SWAPOUTOFRANGELIST
 0000:0028D       O1_OVERLAPBLOCKLIST
 0000:0027D       O1_OUTOFSAMPLESLIST
 0000:0026D       O1_LONGMESSAGELIST
 0000:0025D       O1_PATTERNSIZEMISMATCHLIST
 0000:0024D       O1_OUTOFMEMORYLIST
 0000:0023D       O1_OUTOFSOUNDCARDMEMORYLIST
 0000:0022D       O1_NOBLOCKMARKEDLIST
 0000:0011C       O1_SETPATTERNLENGTH
 0000:000E8       O1_PECONFIGLIST
 0000:000D4       O1_PATTERNEDITLIST
 0000:000BE       O1_HELPLIST
 0000:0001E       O1_ORDERPANNINGLIST
 0000:00000       O1_AUTODETECTLIST
 3D02:00326       GETTIMERCOUNTER
 3D02:00317       STARTCLOCK
 3D02:00264       SETINFOLINE2
 3D02:0024E       SETINFOLINE
 3D02:00243       CLEARINFOLINE
 3D02:00227       IDLEUPDATEINFOLINE
 3D02:00152       UPDATEINFOLINE
 3D02:0012C       UNINITTIMERHANDLER
 3D02:00110       INITTIMERHANDLER
 3D02:000F8       SHOWUSAGETIME
 3D34:0865E       NETWORK_SENDSONGDATAINFORMATION
 3D34:08647       NETWORK_SENDINSTRUMENTHEADER
 3D34:08630       NETWORK_SENDSAMPLEHEADER
 3D34:08613       NETWORK_ENSURENONETWORK
 3D34:085EF       NETWORK_UPDATEPATTERN
 3D34:085DA       NETWORK_UPDATEPATTERNIFIDLE
 3D34:085C9       NETWORK_ADDWORDTOQUEUE
 3D34:084D6       NETWORK_QUEUESAMPLEDATA
 3D34:08496       NETWORK_FINISHEDSENDQUEUE
 3D34:0846A       NETWORK_GETSENDQUEUE
 3D34:07D7B       NETWORK_SHUTDOWN
 3D34:07D45       NETWORK_POLL
 3D34:07BD5       NETWORK_POSTDRIVERSCREEN
 3D34:07B7F       NETWORK_PREDRIVERSCREEN
 3D34:07B02       NETWORK_DRAWDRIVERSCREEN
 3D34:07A63       NETWORK_DRIVERSCREEN
 3D34:07712       D_SLOWINSTRUMENTSORT
 3D34:07670       D_SLOWSAMPLESORT
 3D34:0755A       D_DRAWTIMER
 3D34:074FC       D_POSTTIMERLIST
 3D34:07451       D_SHOWTIME
 3D34:07420       D_RESETTIMER
 3D34:0741A       D_GETFILENAME
 3D34:07416       D_SETDRIVEDIRECTORYFAR
 3D34:0740D       D_RESTOREPRESHELLDIRECTORY
 3D34:073FE       D_GETPRESHELLDIRECTORY
 3D34:06B60       D_VIEWINSTRUMENT
 3D34:06B4F       D_POSTLOADINSTRUMENT
 3D34:06B22       D_PRELOADINSTRUMENT
 3D34:069D1       D_DRAWLOADINSTRUMENT
 3D34:0696A       D_LOADINSTRUMENTNAMES
 3D34:0684F       D_INITLOADINSTRUMENTS
 3D34:0676E       D_DISABLEFILECOLOURS
 3D34:06768       D_GETFORMATTYPE
 3D34:06753       D_CLEARFILENAME
 3D34:065AE       D_DRAWWAVEFORM
 3D34:06403 idle  D_DELETESAMPLEFILE
 3D34:062BC       D_SAVEINSTRUMENT
 3D34:0620D       D_SAVEST3SAMPLE
 3D34:06166       D_SAVERAWSAMPLE
 3D34:06100       D_SAVESAMPLE
 3D34:0607A       D_SAVESONG
 3D34:06049       D_LSCHECKSUSLOOPVALUES
 3D34:06018       D_LSCHECKLOOPVALUES
 3D34:05FB5       LSWINDOW_DOWN
 3D34:05FA1       LSWINDOW_UP
 3D34:050BA       D_SAVEDIRECTORYCONFIGURATION
 3D34:050AF       D_GOTOSTARTINGDIRECTORY
 3D34:0509B       D_GETLOADSAMPLEVARS
 3D34:05037       D_LOADSAMPLENAMES
 3D34:047A9       D_LIPOSTDRIVEWINDOW
 3D34:04787       D_LIPREDRIVEWINDOW
 3D34:04750       D_LIDRAWDRIVEWINDOW
 3D34:0473F       D_LSPOSTDRIVEWINDOW
 3D34:0471B       D_LSPREDRIVEWINDOW
 3D34:046C7       D_LSDRAWDRIVEWINDOW
 3D34:046B7       D_POSTVIEWSAMPLELIBRARY
 3D34:0462D       D_POSTLOADSAMPLEWINDOW
 3D34:045FE       D_PRELOADSAMPLEWINDOW
 3D34:04355       D_DRAWLOADSAMPLEWINDOW
 3D34:040E4       D_INITLOADSAMPLES
 3D34:03AD6       D_SAVES3M
 3D34:03617       D_SAVEIT
 3D34:0347B       D_SAVEMODULE
 3D34:03466       D_CLEARFILESPECIFIER
 3D34:0344A       D_NEWDIRECTORY
 3D34:033BB       D_NEWSPECIFIER
 3D34:033AA       D_POSTSAVEDRIVEWINDOW
 3D34:03399       D_POSTDRIVEWINDOW
 3D34:03321       D_POSTDIRECTORYWINDOW
 3D34:03298 idle  D_POSTFILEWINDOW
 3D34:0322D       D_POSTFILELOADWINDOW
 3D34:031EE       D_POSTFILESAVEWINDOW
 3D34:02EC0       D_LOADIT
 3D34:02C3D       D_LOADMOD
 3D34:02ADC       D_LOAD669
 3D34:0283A       D_LOADS3M
 3D34:0259C       D_LOADMTM
 3D34:0214E       D_LOADXM
 3D34:018EE       D_PREDRIVEWINDOW
 3D34:018C8       D_PREDIRECTORYWINDOW
 3D34:01889       D_PREFILEWINDOW
 3D34:01858       D_LOADSONGNAMES
 3D34:0173D       D_DRAWDRIVEWINDOW
 3D34:016CD       D_DRAWDIRECTORYWINDOW
 3D34:014B0       D_DRAWFILEWINDOW
 3D34:01469       D_INITLOADMODULE
 3D34:01292       D_UNINITDISK
 3D34:010A6       D_INITDISK
 3D34:00F34       DISKOPTIONS
 3D34:002AB       SAMPLENAME
 3D34:00264       INSTRUMENTDIRECTORY
 3D34:0021E       SAMPLEDIRECTORY
 3D34:001D8       SONGDIRECTORY
 3D34:000C4       FILESPECIFIER
 3D34:00066       FILENAME
 3D34:00010       DISKDATAAREA
 459B:00CE5       S_INVERTCURSOR
 459B:00CA5       S_DEFINEHIASCII
 459B:00C84       S_USEPRESETPALETTE
 459B:00C7E       S_GETPALETTEOFFSET
 459B:00C62       S_DRAWSMALLBOX
 459B:00BE2       S_GENERATECHARACTERS
 459B:00BD9       S_GETGENERATIONTABLEOFFSET
 459B:00ABD       S_DRAWSTRING
 459B:00AA8       S_DIRECTDRAWSTRING
 459B:00A99       S_HILIGHT
 459B:00A59       S_SETDIRECTMODE
 459B:009F8       S_UPDATESCREEN
 459B:0098A       S_DRAWBOX
 459B:00975       S_CLEARSCREEN
 459B:00960       S_GETDESTINATION
 459B:0094F       S_UNINITSCREEN
 459B:008B7       S_DEFINESMALLNUMBERS
 459B:00871       S_REDEFINECHARACTERS
 459B:0084B       S_RESETSEQUENCER
 459B:00825       S_SETSEQUENCER
 459B:007FD       S_SETPALETTE
 459B:007F9       S_SETPALETTE2
 459B:0078C       S_RESTORESCREEN
 459B:0076A       S_SAVESCREEN
 459B:006B7       S_INITSCREEN
 459B:006A5       VGAFLAGS
 459B:006A3       CHARACTERGENERATIONOFFSET
 459B:00028       PALETTEDEFS
 466D:00EE2       FORCEMOUSERESTORE
 466D:00EDA       CMDLINEDISABLEMOUSE
 466D:00E8D       SETMOUSECURSORTYPE
 466D:00E86       MOUSEUPDATEDISABLE
 466D:00E7F       MOUSEUPDATEENABLE
 466D:00E78       NEWCHARACTERSET
 466D:00E73       MOUSEGETSTATUS
 466D:00E6A       MOUSEREMOVEEVENTS
 466D:00E61       MOUSECLEAREVENTS
 466D:00E3D       MOUSEADDEVENT
 466D:00DF5       MOUSEINPUT
 466D:00DCA       ADDMOUSEQUEUE
 466D:00DC5       GETKEYBOARDLOCK
 466D:00DC0       SETKEYBOARDLOCK
 466D:00D9B       MOUSERESTOREEVENTS
 466D:00D76       MOUSESAVEEVENTS
 466D:00D27       MOUSESETXY
 466D:00CF8       MOUSETOGGLE
 466D:00CF1       MOUSESECONDSETDISABLE
 466D:00CEA       MOUSESECONDSETENABLE
 466D:00CE5       UNINITMOUSE
 466D:00C8F       INITMOUSE
 466D:00B86       DRAWMOUSE
 466D:00922       RESTOREMOUSEGRAPHICS
 466D:008C8       RESTOREMOUSE
 466D:00000       MOUSECHARACTERGENERATIONOFFSET
 475C:00363       M_OBJECT1LIST
 475C:00360       M_OBJECT1LISTDEFAULT
 475C:00169       M_FUNCTIONHANDLER
 475C:000F1       M_FUNCTIONDIVIDER
 475C:000F0       RELEASETIMESLICE
 4793:00B0F       DOSSHELL
 4793:00AF2       REFRESH
 4793:00ACB       GETENVIRONMENT
 4793:00A9F       CRASHRECOVERY
 4793:00A28       GETSTARTUPKEYLIST
 4793:00A23       ISSTARTUPKEYLIST
 4793:009C5       QUIT
 484B:0597F       PE_NEWPATTERN
 484B:05966       PE_RESTORECURRENTPATTERN
 484B:05948       PE_SAVECURRENTPATTERN
 484B:05940       PE_SETPATTERNMODIFIED
 484B:058FC       PE_RESTOREMIDINOTE
 484B:058C0       PE_TRANSLATEMIDI
 484B:056C4       MIDI_SETINSTRUMENT
 484B:05643       PERESETMODIFIED
 484B:05625       PECHECKMODIFIED
 484B:05577       PEFUNCTION_POSTUNDO
 484B:0555A       PEFUNCTION_PREUNDO
 484B:05524       PEFUNCTION_DRAWUNDO
 484B:054EB idle  PE_CLEARUNDOBUFFER
 484B:0543D       PE_GETPATTERNCONFIGOFFSET
 484B:05372       PE_F7
 484B:052FE       PE_SHOWORDER
 484B:051ED       PE_UPDATEINSTRUMENTS
 484B:0513F       PE_DELETEINSTRUMENT
 484B:0508C       PE_INSERTINSTRUMENT
 484B:04FC4       PE_SWAPINSTRUMENTS
 484B:04FBC       PE_GETLASTINSTRUMENT
 484B:046A4       PE_GETCURRENTPATTERN
 484B:042D9       PE_TRANSLATES3MPATTERN
 484B:041C6       PE_TRANSLATE669PATTERN
 484B:0414C       PE_TRANSLATEMODPATTERN
 484B:040EC       PE_TRANSLATEMTMPATTERN
 484B:03E98       PE_TRANSLATEXMPATTERN
 484B:03A97       PE_GOTOPATTERN
 484B:03A6D       PEFUNCTION_STORECURRENTPATTERN
 484B:031B4       PEFUNCTION_OUTOFMEMORYMESSAGE
 484B:02A4C       PE_SETCOMMANDCURSOR
 484B:02779       PEFUNCTION_INCREASEOCTAVE
 484B:02769       PEFUNCTION_DECREASEOCTAVE
 484B:01D00       PE_POSTPATTERNEDIT
 484B:01B41       PE_PREPATTERNEDIT
 484B:01673       PE_DRAWPATTERNEDIT
 484B:015DB       PE_INITPATTERNEDIT
 484B:015A4       PE_UNINITPATTERNEDIT
 484B:013BA       PE_POSTORDERLIST
 484B:01376       PE_PREORDERLIST
 484B:012E6       PE_DRAWORDERLIST
 484B:012C9       PE_FILLSPEEDTEMPO
 484B:011E0       PE_FILLHEADER
 484B:011B9       PE_GETMAXPATTERN
 484B:0114E       PE_RESETORDERPATTERN
 484B:0109C       PE_GETMAXORDER
 484B:01054       PE_CONVAX2NUM
 484B:00FEF       LASTINSTRUMENT
 484B:00D7D       FLAGS
 484B:00D7B       FASTVOLUMEAMPLIFICATION
 484B:00D7A       MIDICENTRALNOTE
 484B:00D79       MIDIAMPLIFICATION
 484B:00D78       CENTRALISECURSOR
 484B:00D77       COMMANDTOVALUE
 484B:00CA9       ROWHILIGHT2
 484B:00CA8       ROWHILIGHT1
 484B:0087E       PATTERNLENGTHEND
 484B:0087C       PATTERNLENGTHSTART
 484B:0087A       PATTERNSETLENGTH
 484B:0060C       PATTERNMODIFIED
 484B:0060B       MODIFIED
 484B:002D8       AMPLIFICATION
 484B:00086 idle  LASTKEYBOARD1
 484B:00034       MULTICHANNELINFO
 484B:00032       SKIPVALUE
 484B:00030       BASEOCTAVE
 484B:00026       NUMBEROFROWS
 484B:00024       MAXROW
 484B:0001E       PATTERNNUMBER
 484B:0001A       ORDER
 484B:0000A       PATTERNDATAAREA
 4DE4:0D56C       MUSIC_TOGGLESOLOSAMPLE
 4DE4:0D561       MUSIC_TOGGLESOLOINSTRUMENT
 4DE4:0D54C       MUSIC_TOGGLEORDERUPDATE
 4DE4:0D546       MUSIC_GETMIDIDATAAREA
 4DE4:0D51D       MUSIC_SAVEMIDICONFIG
 4DE4:0D518       MUSIC_GETPATTERNLENGTH
 4DE4:0D4FA       MUSIC_SHOWTIME
 4DE4:0D421       MUSIC_TIMESONG
 4DE4:0D3B5       MUSIC_GETDELAY
 4DE4:0D3AF       MUSIC_SETNEXTORDER
 4DE4:0D3AA       MUSIC_SETDRIVERVARIABLE
 4DE4:0D3A5       MUSIC_GETDRIVERVARIABLE
 4DE4:0D3A0       MUSIC_GETDRIVERSCREEN
 4DE4:0D37C       MUSIC_GETLASTCHANNEL
 4DE4:0D360       MUSIC_INITMIXTABLE
 4DE4:0D35B       MUSIC_PATTERNSTORAGE
 4DE4:0D347       MUSIC_TOGGLEREVERSE
 4DE4:0D341       MUSIC_GETPITCHTABLE
 4DE4:0D33C       MUSIC_GETNUMCHANNELS
 4DE4:0D336       MUSIC_GETFREESOUNDCARDMEMORY
 4DE4:0D2E5       MUSIC_SOUNDCARDLOADALLSAMPLES
 4DE4:0D2CE       MUSIC_SOUNDCARDLOADSAMPLE
 4DE4:0D298       MUSIC_REGETLOOPINFORMATION
 4DE4:0D27F       MUSIC_DECREASEVOLUME
 4DE4:0D263       MUSIC_INCREASEVOLUME
 4DE4:0D25C       MUSIC_REVERSECHANNELS
 4DE4:0D256       MUSIC_SETLIMIT
 4DE4:0D1D6       MUSIC_ASSIGNSAMPLETOINSTRUMENT
 4DE4:0D1C5       MUSIC_GETDISPLAYVARIABLES
 4DE4:0D1BF       MUSIC_SETADDRESS
 4DE4:0D1B9       MUSIC_SETIRQ
 4DE4:0D1B3       MUSIC_SETMIXSPEED
 4DE4:0D1AC       MUSIC_SETDMA
 4DE4:0D1A1       MUSIC_SETSOUNDCARDDRIVER
 4DE4:0D17E       MUSIC_SETSOUNDCARD
 4DE4:0D165       MUSIC_DECREASESPEED
 4DE4:0D14C       MUSIC_INCREASESPEED
 4DE4:0D134       MUSIC_INITSTEREO
 4DE4:0D115       MUSIC_INITMUTETABLE
 4DE4:0D0B1       MUSIC_SOLOCHANNEL
 4DE4:0D0AA       MUSIC_UNMUTEALL
 4DE4:0D079       MUSIC_TOGGLECHANNEL
 4DE4:0D006       MUSIC_SETGLOBALVOLUME
 4DE4:0CFCA       MUSIC_LASTORDER
 4DE4:0CF9E       MUSIC_NEXTORDER
 4DE4:0CF95       MUSIC_GETSLAVECHANNELINFORMATIONTABLE
 4DE4:0CF8F       MUSIC_GETHOSTCHANNELINFORMATIONTABLE
 4DE4:0CF39       MUSIC_PLAYSAMPLE
 4DE4:0CEB7       MUSIC_PLAYNOTE
 4DE4:0CEAF       MUSIC_UPDATEPATTERNOFFSET
 4DE4:0CDC0       MUSIC_STOP
 4DE4:0CD6D       MUSIC_KBPLAYSONG
 4DE4:0CD2C       MUSIC_PLAYPARTSONG
 4DE4:0CCF5       MUSIC_PLAYSONG
 4DE4:0CCCB       MUSIC_PLAYPATTERN
 4DE4:0CCB2       MUSIC_GETPLAYMODE2
 4DE4:0CC9A       MUSIC_GETPLAYMODE
 4DE4:0CC22       MUSIC_GETSAMPLELOCATION
 4DE4:0CBEC       MUSIC_GETNUMBEROFINSTRUMENTS
 4DE4:0CBC4       MUSIC_GETNUMBEROFSAMPLES
 4DE4:0C254       MUSIC_GETINSTRUMENTMODE
 4DE4:0C232       MUSIC_SHOWAUTODETECTSOUNDCARD
 4DE4:0C17E       MUSIC_AUTODETECTSOUNDCARD
 4DE4:0C082       MUSIC_GETSONGSEGMENT
 4DE4:0C061       MUSIC_UNINITMUSIC
 4DE4:0C056       MUSIC_CLEARALLINSTRUMENTS
 4DE4:0C034       MUSIC_CLEARINSTRUMENT
 4DE4:0C023       MUSIC_RELEASEALLPATTERNS
 4DE4:0C012       MUSIC_RELEASEALLSAMPLES
 4DE4:0C001       MUSIC_CLEARALLSAMPLENAMES
 4DE4:0BFDE       MUSIC_CLEARSAMPLENAME
 4DE4:0BF62       MUSIC_RELEASESAMPLE
 4DE4:0BEA5       MUSIC_ALLOCATESAMPLE
 4DE4:0BDDD       MUSIC_ALLOCATEPATTERN
 4DE4:0BD89       MUSIC_GETPATTERNLOCATIONNOCOUNT
 4DE4:0BD80       MUSIC_GETPATTERNLOCATION
 4DE4:0BD38       MUSIC_GETPATTERN
 4DE4:0BCF4       MUSIC_RELEASEPATTERN
 4DE4:0BCAF       MUSIC_INITMUSIC
 4DE4:0BC9F       MUSIC_REINITSOUNDCARD
 4DE4:0BC61       MUSIC_POLL
 4DE4:0BC51       MUSIC_GETWAVEFORM
 4DE4:09966       MIDIDATAAREA
 4DE4:09964       SONGDATAAREA
 4DE4:00352       CURRENTPATTERN
 5B40:0048C       GLBL_DRIVERSCREEN
 5B40:00479       GLBL_TIMERSCREEN
 5B40:00411       GLBL_RESTOREMODE
 5B40:003ED       GLBL_SAVEMODE
 5B40:003DA       GLBL_RIGHTSQUAREBRACKET
 5B40:003C7       GLBL_LEFTSQUAREBRACKET
 5B40:003B4       GLBL_RIGHTBRACE
 5B40:003A1       GLBL_LEFTBRACE
 5B40:00395       GLBL_ALT_F8
 5B40:00389       GLBL_ALT_F7
 5B40:0037D       GLBL_ALT_F6
 5B40:00371       GLBL_ALT_F5
 5B40:00365       GLBL_ALT_F4
 5B40:00359       GLBL_ALT_F3
 5B40:0034D       GLBL_ALT_F2
 5B40:00341       GLBL_ALT_F1
 5B40:0033C       GLBL_GETCURRENTMODE
 5B40:00337       GLBL_SETCURRENTMODE
 5B40:00300       GLBL_GETHEADERMODE
 5B40:002ED       GLBL_CTRL_F12
 5B40:002DD       GLBL_CTRL_F5
 5B40:002C5       GLBL_CTRL_F4
 5B40:002AD       GLBL_CTRL_F3
 5B40:0029A       GLBL_CTRL_F1
 5B40:00287       GLBL_F12
 5B40:0025E       GLBL_F11_2
 5B40:00256       GLBL_F11
 5B40:00231       GLBL_F10
 5B40:00211       GLBL_F9
 5B40:00208       GLBL_F8
 5B40:001F2       GLBL_SHIFT_F6
 5B40:001DA       GLBL_SHIFT_F9
 5B40:001C7       GLBL_SHIFT_F1
 5B40:001AF       GLBL_LOADINSTRUMENT
 5B40:00197       GLBL_LOADSAMPLE
 5B40:00182       GLBL_F6
 5B40:00132       GLBL_F5
 5B40:00112       GLBL_F4_2
 5B40:000F4       GLBL_F4
 5B40:000DC       GLBL_F3
 5B40:00074       GLBL_F2_2
 5B40:00069       GLBL_F2
 5B40:00003       CURRENTMODE
 5B89:01E9A       FOURIER_POSTFUNCTION
 5B89:01E96       FOURIER_IDLELIST
 5B89:01DA5       FOURIER_DRAWSCREEN
 5B89:01DA2       FOURIER_PREDRAWSCREEN
 5B89:01D40       FOURIER_START
 5B89:01C8A       FOURIER_CHANGEPALETTE
 5B89:01BB1       FOURIER_TRANSFORM
 5B89:01B86       FOURIER_CREATETABLE
 5B89:01B11       DISPLAY_SELECTDISPLAYLIST
 5B89:01AAC       DISPLAY_GETDISPLAYWINDOWDATA
 5B89:01A40       DISPLAYUPDATESCREEN
 5B89:01881       DISPLAYMINUS
 5B89:01878       DISPLAYPLUS
 5B89:0184A       POSTDISPLAYDATA
 5B89:0179F       DRAWDISPLAYDATA
 5D73:003F7       E_GETINTERNALEMSHANDLE
 5D73:003F2       E_GETEMSVERSION
 5D73:003DC       E_RESTOREEMSPAGEFRAME
 5D73:003C1       E_SAVEEMSPAGEFRAME
 5D73:003BA       E_EMSAVAILABLE
 5D73:00374       E_ALLOCATEEMS
 5D73:002E7       E_RELEASEBLOCKEMS
 5D73:001FD       E_ALLOCATEBLOCKEMS
 5D73:001DA       E_MAPALIGNEDBLOCKEMS
 5D73:001D5       E_GETEMSPAGEFRAME
 5D73:001C4       E_UNINITEMS
 5D73:0019B       E_MAPEMSMEMORY
 5D73:00180       E_MAPAVAILABLEEMSMEMORY
 5D73:00109       E_RELEASEEMS
 5D73:000EB       E_GETFREEEMS
 5D73:0002A       E_INITEMS
 5DB2:001AA       ERROR_UNINITHANDLER
 5DB2:0018F       ERROR_INITHANDLER
 5DCD:0368C       I_GETPRESETENVELOPEOFFSET
 5DCD:03675       I_SAMPLEBUTTONHANDLER
 5DCD:03671       UPDATEWAVEFORM
 5DCD:03635       I_IDLEUPDATEENVELOPE
 5DCD:035E3       I_POSTPITCHPANCENTER
 5DCD:035D3       I_PREPITCHPANCENTER
 5DCD:035A1       I_DRAWPITCHPANCENTER
 5DCD:03589       I_TOGGLEMULTICHANNEL
 5DCD:0353D       I_DECREASEPLAYCHANNEL
 5DCD:03522       I_INCREASEPLAYCHANNEL
 5DCD:03505       I_PLAYSAMPLE
 5DCD:034D8       MIDI_PLAYSAMPLE
 5DCD:034D1       I_TAGSAMPLE
 5DCD:034CA       I_TAGINSTRUMENT
 5DCD:034BD       I_CLEARTABLES
 5DCD:0343E       I_SHOWINSTRUMENTPLAY
 5DCD:033F2       I_SHOWSAMPLEPLAY
 5DCD:033D6       I_INSTRUMENTLISTNOTEOFF
 5DCD:033A9       I_INSTRUMENTLISTSPACE
 5DCD:02B39       I_MAPENVELOPE
 5DCD:02A8D       I_POSTENVELOPE
 5DCD:02A85       I_PREENVELOPE
 5DCD:029F5       I_DRAWENVELOPE
 5DCD:02966       I_UPDATEINSTRUMENT
 5DCD:02917       I_SWAPINSTRUMENTS
 5DCD:028EF       I_COPYINSTRUMENT
 5DCD:028A5       I_SCALEINSTRUMENTVOLUMES
 5DCD:0285B       I_SCALESAMPLEVOLUMES
 5DCD:0282E       I_REPLACEINSTRUMENT
 5DCD:02813       I_SAMPLESPEEDSEMIDOWN
 5DCD:027F2       I_SAMPLESPEEDSEMIUP
 5DCD:027E1       I_HALVESAMPLESPEED
 5DCD:027C1       I_DOUBLESAMPLESPEED
 5DCD:02781       I_EXCHANGEINSTRUMENTS
 5DCD:02437       I_POSTNOTEWINDOW
 5DCD:023FB       I_PRENOTEWINDOW
 5DCD:0233F       I_DRAWNOTEWINDOW
 5DCD:021EA       I_POSTINSTRUMENTWINDOW
 5DCD:02157       I_PLAYNOTE
 5DCD:0210F       MIDI_PLAYNOTE
 5DCD:020E2       MIDI_NOTEOFF
 5DCD:020CD       MIDI_CLEARTABLE
 5DCD:020C3       MIDI_FINDCHANNEL
 5DCD:020BB       MIDI_GETCHANNEL
 5DCD:0207B       MIDI_ALLOCATECHANNEL
 5DCD:02035       I_PREINSTRUMENTWINDOW
 5DCD:01F7A       I_DRAWINSTRUMENTWINDOW
 5DCD:01DA6       I_TOGGLESAMPLEQUALITY
 5DCD:01BEE       I_REVERSESAMPLE
 5DCD:01AB6       I_AMPLIFYSAMPLE
 5DCD:019CF       I_CENTERSAMPLE
 5DCD:01972       I_RESIZESAMPLENOINT
 5DCD:0196A       I_RESIZESAMPLE
 5DCD:016A0       I_REPLACESAMPLE
 5DCD:0161C       I_SWAPSAMPLES
 5DCD:015D7       I_EXCHANGESAMPLES
 5DCD:01372 idle  I_CLEARSAMPLENAME
 5DCD:01320       I_CUTSAMPLE
 5DCD:0124F       I_CUTSAMPLEBEFORELOOP
 5DCD:011DC       I_INVERTSAMPLE
 5DCD:01174       I_CONVERTSAMPLE
 5DCD:01131       I_DELETEINSTRUMENT
 5DCD:0111A       I_PRINTC5FREQUENCY
 5DCD:01116       I_CALCULATEC5SPEED
 5DCD:010DE       I_DELETESAMPLE
 5DCD:00F09       I_DRAWWAVEFORM
 5DCD:00ECB       I_CHECKSUSLOOPVALUES
 5DCD:00E8D       I_CHECKLOOPVALUES
 5DCD:00E25       I_SHOWSAMPLEINFO
 5DCD:00D7A       I_SAMPLEUP
 5DCD:00D5D       I_SAMPLEDOWN
 5DCD:00BC3       I_POSTSAMPLELIST
 5DCD:00B68       I_PRESAMPLELIST
 5DCD:00A71       I_DRAWSAMPLELIST
 5DCD:009C2       I_SELECTSCREEN
 5DCD:0099A       I_GETSAMPLEOFFSET
 5DCD:00987       I_GETINSTRUMENTOFFSET
 5DCD:00981       I_GETINSTRUMENTSCREEN
 5DCD:00145       SAMPLEAMPLIFICATION
 5DCD:0013D       INSTRUMENTEDIT
 5DCD:00135       NODEHELD
 5DCD:00127       MAXNODE
 5DCD:00121       NEWSAMPLESIZE
 5DCD:0011D       SAMPLENUMBERINPUT
 5DCD:00011       SAMPLENUMBER
 5DCD:0000E       INSTRUMENTSCREEN
 5DCD:0000C       INSTRUMENTAMPLIFICATION
 6136:01DDC       F_MIDI_PGDN
 6136:01DC4       F_MIDI_PGUP
 6136:01DB2       F_MIDI_DOWN
 6136:01D99       F_MIDI_UP
 6136:01D72       F_SHOWMIDIZXXINPUT
 6136:01D5B       F_FILEQUIT
 6136:01D44       F_FILEDOSSHELL
 6136:01D32       F_FILESAVEAS
 6136:01D1B       F_FILESAVECURRENT
 6136:01D06       F_FILENEW
 6136:01CF4       F_FILELOAD
 6136:01CE0       F_FILEMENU
 6136:01CCE       F_SAMPLELIBRARY
 6136:01CBC       F_RELOADGRAVIS
 6136:01CAA       F_INSTRUMENTLIBRARY
 6136:01C98       F_INSTRUMENTLIST
 6136:01C86       F_SAMPLELIST
 6136:01C72       F_INSTRUMENTMENU
 6136:01C5E       F_SAMPLEMENU
 6136:01C4C       F_DRIVERSCREEN
 6136:01C35       F_CALCULATELENGTH
 6136:01C23       F_REINITSOUNDCARD
 6136:01C11       F_STOP
 6136:01BFF       F_PLAYMARK
 6136:01BED       F_PLAYORDER
 6136:01BDB       F_PLAYPATTERN
 6136:01BC9       F_PLAYSONG
 6136:01BB7       F_INFOPAGE
 6136:01BA3       F_PLAYBACKMENU
 6136:01B91       F_HELP
 6136:01B84       F_MESSAGEEDITOR
 6136:01B77       F_VIEWORDERPAN
 6136:01B6A       F_VIEWVARIABLES
 6136:01B5D       F_VIEWPATTERN
 6136:01B44       F_MAINMENU
 6136:01A9E       F_NEWSONG
 6136:01A96       F_RESET5NUMINPUTPOS
 6136:01A86       F_SETAMIGA
 6136:01A76       F_SETLINEAR
 6136:01A61       F_SETMONO
 6136:01A4C       F_SETSTEREO
 6136:019DF       F_SETCONTROLINSTRUMENT
 6136:019CF       F_SETCONTROLSAMPLE
 6136:0195C       F_CONFIGBUTTONSETUP
 6136:0191D       F_DRAWSMCCHANNELS
 6136:018B8       F_DRAWHEADER
 6136:01798       F_POST5NUM
 6136:01779       F_PRE5NUM
 6136:01700       F_DRAW5NUM
 6136:015B1       F_POST3NUM
 6136:01592       F_PRE3NUM
 6136:01518       F_DRAW3NUM
 6136:013EF       F_POSTTOGGLE
 6136:013BC       F_PRETOGGLE
 6136:01346       F_DRAWTOGGLE
 6136:010E1       F_GOTOEMPTYLIST
 6136:0102A       F_POSTSTRINGINPUT
 6136:01006       F_PRESTRINGINPUT
 6136:00F92       F_DRAWSTRINGINPUT
 6136:00EDD       F_RETURN1
 6136:00DF9       F_RETURN192
 6136:00DF2       F_RETURN64
 6136:00DEC       F_RETURN0
 6136:00DE8       F_REDRAWSCREEN
 6136:00DA6       F_SHOWCHANNELS
 6136:00D61       F_DRAWINFOLINE
 6136:00B6E       F_POSTTHUMBBAR
 6136:00B22       F_POSTSCALABLETHUMBBAR
 6136:00A71       F_PRESCALABLETHUMBBAR
 6136:009BF       F_PRETHUMBBAR
 6136:008D6       F_DRAWSCALABLETHUMBBAR
 6136:0080B       F_DRAWTHUMBBAR
 6136:00505       F_POSTBUTTONOBJECT
 6136:004CC       F_PREBUTTONOBJECT
 6136:00427       F_DRAWBUTTONOBJECT
 6136:003E0       F_CHARACTERDEFINITIONS
 6136:003D8       F_SETDIRECTMODE
 6136:003C8       F_POSTEXITOBJECT
 6136:00383       F_DRAWTEXTOBJECT
 6136:0036D       F_DRAWBOXOBJECT
 6136:00369       F_CALLFARFUNCTION
 6136:00363       F_CALLFARPOSTFUNCTION
 6136:0035F       F_CALLFARPREFUNCTION
 6136:00344       F_INSTRUMENTBUTTONHANDLER
 6136:00341       F_NOTHING
 6136:000D8       THUMBSTRINGENTER
 6315:0238C       H_SETHELPCONTEXT
 6315:02377       H_HELPESC
 6315:0236D       H_HELPPGDN
 6315:0235A       H_HELPPGUP
 6315:0232F       H_HELPDOWN
 6315:0231F       H_HELPUP
 6315:022FD       H_HELP
 6315:0228C       H_DRAWHELP
 654E:00ABD       MIDISEND
 654E:00AB6       MIDIBUFFEREMPTY
 654E:00AAD       K_SETSCROLLLOCK
 654E:00A9B       K_REMOVEKEYBOARDTYPE
 654E:00A46       K_INSTALLKEYBOARDTYPE
 654E:00A23       K_SHOWMIDIINPUT
 654E:009A6       K_DRAWTABLES
 654E:00996       K_RESETKEYBOARDTABLES
 654E:0098F       K_ISKEYDOWN
 654E:00977       K_ISANYKEYDOWN
 654E:00966       K_CLEARKEYBOARDQUEUE
 654E:0070B       K_GETKEY
 654E:006D7       K_ISKEYWAITING
 654E:006B3       K_UNINSTALLDOSHANDLER
 654E:00693       K_INSTALLDOSHANDLER
 654E:00651       K_UNINITKEYBOARD
 654E:005EA       K_INITKEYBOARD
 65FE:0006F       MMTSR_UNINSTALLMMTSR
 65FE:00001       MMTSR_INSTALLMMTSR
 6681:02392       MSG_GETMESSAGEOFFSET
 6681:0237D       MSG_GETMESSAGELENGTH
 6681:020BE       MSG_POSTMESSAGE
 6681:0208F       MSG_PREMESSAGE
 6681:01FE5       MSG_DRAWMESSAGE
 6681:01FCB       MSG_RESETMESSAGE
 68BB:0025B       VESA_SETBLOCK
 68BB:00244 idle  VESA_GETINFO
 68BB:00221       VESA_SETMODE
 68BB:00201       VESA_DETECT

Program entry point at 4793:0637

